:100000000AC0EAC113C221C020C01FC039C22DC01E
:100010001CC01BC01AC011241FBECFEDCDBF10E005
:10002000A0E6B0E0E2E3F5E003C0C89531960D929A
:10003000A036B107D1F710E0A0E6B0E001C01D92F4
:10004000A036B107E1F759D272C2DACF8CB95E9B04
:10005000FECF5E9A08955F9BFECF5F988CB10895A6
:1000600084E489B988E18AB908951F920F920FB686
:100070000F9211248F938FE48CB95E9BFECF5E9A12
:100080008BE48CB95E9BFECF5E9A80E28CB95E9B5E
:10009000FECF5E9A8CB18CB95E9BFECF5E9A8AE0F1
:1000A0008CB95E9BFECF5E9A8F910F900FBE0F9022
:1000B0001F90189589E48CB95E9BFECF5E9A8FE401
:1000C0008CB95E9BFECF5E9A80E28CB95E9BFECFC0
:1000D0005E9A83E48CB95E9BFECF5E9A81E68CB912
:1000E0005E9BFECF5E9A82E78CB95E9BFECF5E9AE6
:1000F00084E78CB95E9BFECF5E9A80E28CB95E9BF2
:10010000FECF5E9A88E28CB95E9BFECF5E9A83E654
:100110008CB95E9BFECF5E9A89E28CB95E9BFECF66
:100120005E9A80E28CB95E9BFECF5E9A82E38CB9C8
:100130005E9BFECF5E9A80E38CB95E9BFECF5E9A9B
:1001400081E38CB95E9BFECF5E9A81E38CB95E9BA6
:10015000FECF5E9A80E28CB95E9BFECF5E9A8CE405
:100160008CB95E9BFECF5E9A85E68CB95E9BFECF16
:100170005E9A85E78CB95E9BFECF5E9A83E68CB96A
:100180005E9BFECF5E9A8FE68CB95E9BFECF5E9A39
:100190008EE68CB95E9BFECF5E9A8FE68CB95E9B35
:1001A000FECF5E9A85E68CB95E9BFECF5E9A80E2BA
:1001B0008CB95E9BFECF5E9A83E58CB95E9BFECFC9
:1001C0005E9A86E28CB95E9BFECF5E9A88E48CB91B
:1001D0005E9BFECF5E9A8AE08CB95E9BFECF5E9AF4
:1001E0008DE08CB95E9BFECF5E9A0895982F85E4D2
:1001F0008CB95E9BFECF5E9A82E78CB95E9BFECF88
:100200005E9A82E78CB95E9BFECF5E9A8FE68CB9D0
:100210005E9BFECF5E9A82E78CB95E9BFECF5E9AB4
:1002200080E28CB95E9BFECF5E9A9CB95E9BFECF4E
:100230005E9A8AE08CB95E9BFECF5E9A8DE08CB9A7
:100240005E9BFECF5E9A08955F9BFECF5F988CB158
:10025000873609F48DC088366CF1833709F44DC0B8
:10026000843751F55F9BFECF5F988CB1803309F0E6
:10027000A7C05F9BFECF5F988CB187FDAAC0809519
:1002800082BF86E083BF82E089BF8FE48CB95E9B2A
:10029000FECF5E9A8BE48CB95E9BFECF5E9A8AE0BD
:1002A0008CB95E9BFECF5E9A8DE08CB95E9BFECFD3
:1002B0005E9A0895843519F080E398DF08955F9B76
:1002C000FECF5F988CB1803309F077C089B78D7FFE
:1002D00089BF8FE48CB95E9BFECF5E9A8BE48CB9AC
:1002E0005E9BFECF5E9A8AE08CB95E9BFECF5E9AE3
:1002F0008DE08CB95E9BFECFDBCF40E020E030E0AC
:1003000061E070E05F9BFECF5F989CB1892F8053C6
:10031000823008F05BC0913309F12F5F3F4F2830E6
:10032000310581F75F9BFECF5F988CB1833709F071
:100330004AC048BB8FE48CB95E9BFECF5E9A8BE4CB
:100340008CB95E9BFECF5E9A8AE08CB95E9BFECF35
:100350005E9A8DE08CB95E9BFECFAACF862F972F39
:10036000022E02C0880F991F0A94E2F7482BD5CFBE
:1003700020E030E050E341E388B390E0022E02C079
:10038000959587950A94E2F780FF13C04CB95E9B60
:10039000FECF5E9A2F5F3F4F2830310569F78AE024
:1003A0008CB95E9BFECF5E9A8DE08CB95E9BFECFD2
:1003B0007FCF5CB95E9BFECFECCF86E317DF08955D
:1003C00085E314DF089583E311DF089582E30EDFF0
:1003D000089584E30BDF08951F920F920FB60F92DA
:1003E00011248F9389E48CB95E9BFECF5E9A8EE4D4
:1003F0008CB95E9BFECF5E9A84E58CB95E9BFECF86
:100400005E9A80E38CB95E9BFECF5E9A8AE08CB9DF
:100410005E9BFECF5E9A8DE08CB95E9BFECF5E9AAE
:100420008F910F900FBE0F901F9018951F920F92F3
:100430000FB60F9211248F9389E48CB95E9BFECF87
:100440005E9A8EE48CB95E9BFECF5E9A84E58CB991
:100450005E9BFECF5E9A81E38CB95E9BFECF5E9A77
:100460008AE08CB95E9BFECF5E9A8DE08CB95E9B74
:10047000FECF5E9A8F910F900FBE0F901F90189530
:100480001F920F920FB60F9211248F9384E58CB9AF
:100490005E9BFECF5E9A89E48CB95E9BFECF5E9A2E
:1004A0008DE48CB95E9BFECF5E9A85E48CB95E9B31
:1004B000FECF5E9A82E58CB95E9BFECF5E9A80E3AA
:1004C0008CB95E9BFECF5E9A8AE08CB95E9BFECFB4
:1004D0005E9A8DE08CB95E9BFECF5E9A89B78D7F68
:1004E00089BF83B78D7F83BF83B78B7F83BF8F9196
:1004F0000F900FBE0F901F901895B89AB99ABA9A9C
:10050000BB9ABC9ABD9ABE9ABF9A8A98929A8B98C7
:10051000939A80EC8BBF8AE085BF18BA84E489B9CE
:1005200088E18AB97894C6DD8FDE8EDEFDCFF8943F
:02053000FFCFFB
:00000001FF
